:020000040000FA
:100000008501FF2383163128CF000308D00010108C
:100010000E08CD000F08CE008F018E0110140C18B1
:10002000BB210C1C3B210C108B1050088300CF0E01
:100030004F0E09008207A828AD28B228B728BC288F
:10004000C128C628CB28D028D5288A018207C62AED
:10005000D12ADC2AE72AF22AFD2A082B132B1E2B91
:10006000292B900020309F00103091000130870034
:100070000430850034309500831207309900073032
:1000800062003530900011309F0062209D200630C4
:10009000B900A220B90B4928192190308B00A10189
:1000A0006400A1186C212118C3210B195A200C18C7
:1000B000BB2150280B11A00A20080D3A031D08008F
:1000C000A00119298D200715792021307620C5300F
:1000D00076200630762013307620203076200C30C3
:1000E000762008000301B60007157D28B600071129
:1000F0007D2887128D208716003487100830B700BE
:100100000712B61B8715B61F87116400071600007B
:10011000B60DB70B80288714003464000730B80090
:1001200064003230BA006400FA30B900B90B962886
:10013000BA0B9328B80B902808008030BB004030E1
:10014000BC00EB285430BA007220BA0BA428080077
:100150000830D1001030D200DA281830D1005830E1
:10016000D200DA282030D1002830D200DA2820301E
:10017000D1003030D200DA283830D1004030D200FF
:10018000DA284830D1003030D200DA284830D100A7
:100190005030D200DA280830D1005830D200DA28A6
:1001A0000830D1005030D200DA280830D100303089
:1001B000D200DA280830D300EB20E4200830D30046
:1001C000BC0AEB205208D1005108EF207320D10A5D
:1001D000D30BE42808003B0876203C08762864000E
:1001E00083169B001C141A08831208000310103099
:1001F000A300A401A501A601A90DA80DA60DA50D9A
:10020000A40DA30B04290800263084000E212530FC
:1002100084000E21243084000E21FC2803300007C6
:10022000A200A219800030300007A200A21B8000AB
:1002300008009F1464009F181A291E08A900A8012D
:10024000F620CC30BB004430BC0026080F391A2001
:10025000C030BB004430BC00260E0F391A2072207B
:10026000C0307320C0307320B630BB004430BC00B7
:1002700025080F391A284908003A031D4229CC01E4
:10028000CB01CA014D08CC07031C4A290310CB0A35
:100290000318CA0A4E08CB070318CA0AC90A490834
:1002A000203A031D0800C901CA0CCB0CCC0CCA0CA7
:1002B000CB0CCC0CCA0CCB0CCC0CCA0CCB0CCC0C85
:1002C000CA0CCB0CCC0C0310AA014B08AB004C0899
:1002D000AC00A114211108007A21F62026080F395C
:1002E000C800260E0F39C70025080F39C600A11017
:1002F000211408002C08003A031D85292B08003A18
:10030000031D8529A901A80100340530B000B830CB
:10031000B100D830B2001830A300A701A801A9018C
:10032000AD01AE01AF010310B20DB10DB00DAF0DB7
:10033000AE0DAD0D2A082D02031DA4292B082E0297
:10034000031DA4292C082F02031CB5292C08AF0279
:10035000031CAE032E08FF3A0319AD032B08AE02AF
:10036000031CAD032A08AD020314A90DA80DA70DA7
:10037000A30B93290800C901C601C701C801211DAB
:1003800021142115080021109D20A220A220A220C6
:10039000A2204608031DD3294708031DD929480870
:1003A000031DDF29E5298330BB004030BC0046082F
:1003B00025209830BB004030BC0047082520AD30D8
:1003C000BB004030BC0048082520C230BB00403094
:1003D000BC0003012528C422A022A222A422952227
:1003E000A422A222A022C42A9122B422A422A222C0
:1003F000A02A9122A622A822AA22C42AC422AA2282
:10040000A822A6229522A622A822AA22C42A9122A4
:10041000A422A222A022C42AA022AC22AE22B02270
:100420000F309622B022AE22AC22A02AC422AA22E9
:10043000B622B222C0309622B222B622AA22C42A02
:10044000C422A022AC22AE2203309622AE22AC22DD
:10045000A022C42AAA22B622B222B822F0309622C2
:10046000B822B222B622AA2A7220BA22BC22BE2206
:100470000F309622B022AE22AC22A02A7220722027
:10048000C022C222C0309622B622AA22C42AC42286
:10049000A022AC22AE22BC2203309622BA227220C5
:1004A0007228AA22B622B222B822F03096229E22C8
:1004B000C222C022722872207220BA22BC220330CB
:1004C0009622AE22AC22A022C42A7220C022C222CE
:1004D0009E22F0309622B822B222B622AA2AA02268
:1004E000A222A422B4229522B422A422A222A02ACB
:1004F0009122A622A822AA22C42AA022AC22AE229D
:10050000B0220F309622BE22BC22BA227228C42208
:10051000AA22B622B222C0309622C222C022722063
:10052000722872207220722072200301B9000A30F2
:10053000BA0039087320BA0B992A0800E0307328F2
:10054000FE307328FC307328F83073281F3073286E
:100550003F3073287F307328FD307328FB307328B9
:10056000F7307328DF307328F0307328BF307328DA
:10057000EF30732801307328033073280730732855
:1005800080307328C0307328FF307328EB200C2292
:10059000BC0AEB20FE21BC0AEB20EB21BC0AEB20BD
:1005A0002A2AEB20F421BC0AEB20F921BC0AEB201B
:1005B0000722BC0AEB20782AEB203422BC0AEB206D
:1005C0003E22BC0AEB204722BC0AEB20512AEB203A
:1005D0003422BC0AEB203E22BC0AEB205B22BC0A80
:1005E000EB20652AEB206F22BC0AEB201622BC0A06
:1005F000EB205B22BC0AEB20782AEB207D22BC0A90
:10060000EB208722BC0AEB205B22BC0AEB20652A88
:10061000EB207D22BC0AEB208722BC0AEB202022A3
:10062000BC0AEB202A2AEB200C22BC0AEB20FE217C
:10063000BC0AEB200722BC0AEB20782AEB200C2214
:10064000BC0AEB201622BC0AEB202022BC0AEB20BD
:100650002A2AEB200C22BC0AEB201622BC0AEB2033
:080660005B22BC0AEB20652AB5
:0207FE000034C5
:02400E008C0123
:104200005500550055005500550055005500550006
:10421000FC00FC000C000C000C000C00FC00FC007E
:10422000FF00FF00C000C000C000C000FF00FF0092
:10423000000000000000000030003000FC00FC0026
:104240000C000C000C000C000C000C00FC00FC002E
:10425000FF00FF00C300C300C300C300C300C300CE
:10426000C300C300C300C300C300C300FF00FF00BE
:10427000FC00FC000000000000000000FC00FC004E
:10428000030003000300030003000300FF00FF001E
:10429000FC00FC000C000C000C000C000C000C00DE
:1042A000FF00FF00C300C300C300C300FF00FF0006
:1042B000000000000000000000000000FF00FF0000
:1042C0005500550055005500550055005500550046
:1042D0005500550055005500550055005500550036
:1042E0005500550055005500550055005500550026
:1042F0005500550055005500550055005500550016
:00000001FF
